:100000000C9434000C9400000C9400000C9400003C
:100010000C9400000C9400000C9400000C94000060
:100020000C9400000C944E010C9400000C94000001
:100030000C9400000C942F010C9400000C94000010
:100040000C9400000C9400000C9489010C94A601FF
:100050000C94BF010C9400000C9400000C94000060
:100060000C9400000C9400000FEF0DBF08E00EBFD1
:100070008FEF90E00E941E0114E01093810015E0C4
:100080001093020111E010936F0078940FE107B90B
:1000900098B90E943E0126E02093030121E02093BD
:1000A000060121E0209370000E9465011091040177
:1000B0001813FCCF90936F0090937000409A0E94A9
:1000C0001E0114E01093810011E01093020111E071
:1000D00010936F000E943E0126E02093030122E06E
:1000E0002093060121E02093700010910401181361
:1000F000FCCF90936F0090937000419A0E941E0174
:1001000014E01093810011E01093020111E01093AC
:100110006F000E943E0126E02093030124E020931B
:10012000060121E02093700090931201A3E2B1E058
:10013000909310013091C10030693093C10030912B
:1001400010013813FCCF3091C1003F743093C100CF
:100150009093C600A0E2B1E0909311016D9160937D
:10016000C6003091C10038623093C1003091110156
:100170003813FCCF3091C10037793093C100909390
:10018000C600A0E0B2E0809312013091C100306956
:100190003093C100309112013913FCCF3091C1006E
:1001A0003F743093C1009093C6001091040118135E
:1001B000FCCF90936F0090937000429A0E941E01B2
:1001C00014E01093810011E01093020111E01093EC
:1001D0006F000E943E0126E02093030128E0209357
:1001E000060121E020937000109104011813FCCF48
:1001F00090936F0090937000439A0E941E0114E048
:100200001093810011E01093020111E010936F0030
:100210000E943E0126E02093030120E12093060185
:1002200021E020937000109104011813FCCF9093EB
:100230006F0090937000449AFFCFF89490938000E1
:100240009093810090938200909385009093840016
:1002500090936F00909300019093040108951F9371
:1002600010910001139570910201171719F41127CD
:1002700080930401109300011F9118959093B00092
:100280009093B1009093B2009093700027E0209378
:10029000B100909305019093010108952F9320914F
:1002A0000101239570910301271759F428B170912A
:1002B0000601272728B920910501209520930501E3
:1002C0002227209301012F9118959093C6009093B7
:1002D000C0009093C1009093C20030E03093C500FD
:1002E00033E33093C40036E03093C20031E43093FE
:1002F000200133E4309321013BE43093220132E5C5
:100300003093230135E43093240131E53093250106
:1003100008953F936091C60030911201381306C0D2
:100320006D93A03459F49093120108C03C91361794
:1003300029F41196A63211F4809310013091C10076
:100340003F7730623093C1003F9118953F933091D1
:10035000C1003F7D34FD03C033FD03C00CC03068D5
:100360000AC06C9130646093C6001196A33219F4F0
:100370008093110100C03093C1003F9118953F93C5
:100380003091C10030623F7B3093C1003F9118959E
:00000001FF
